:10065A002530326264002E350D002E300D003F0623
:0E066A005B4F666D7D077F6F777C395E79711F
:1006B000EF4E60147D737C00ED1D70011CED4C70DD
:0806C000F7EF1F70EB1E80E84C
:0106C800220F
:0606EE0075F00A84AFF074
:0706F400EF90066893FF225E
:1006C900AE07EE1206EE8F27EE75F00A84FE1206CB
:0406D900EE8F262258
:1005A200E4FF74262FF8E6FEE4FDEE3392B4EE2566
:1005B200E0FED2B20000C2B200000DBD08EC0FBFD7
:0A05C20002E0D2B30000C2B3000053
:0105CC00220C
:10063B00C2B57F677E00EF1F70011EEF4E70F7D2C1
:0E064B00B57E007F05EF1F70011EEF4E70F7A9
:01065900227E
:10061800E4FFFE30B5120FEFAC0670010E14D39450
:10062800D0EC940740EDD322A2B5B340FB7F05DFA1
:02063800FEC3FF
:01063A00229D
:1005F400C2B50FBF0000D2B50FBF00000FBF00008F
:10060400A2B592017E007F09EF1F70011EEF4E70AC
:03061400F7A20149
:0106170022C0
:10067800E4FD7C011205F4E433FFC43333335480C2
:0C068800FEEDC3134EFD0CBC09EAAF05EB
:010694002243
:09051A007F017E001206B07FCCC7
:100523007E01EF139201EFC313FF30011BC2B50B22
:10053300BB00000BBB0000D2B57A007B09EB1B703C
:10054300011AEB4A70F7801BC2B57A007B09EB1BDB
:1005530070011AEB4A70F7D2B50BBB00010A0BBB53
:0705630000010A0EBE09BBF6
:01056A00226E
:1006DD0012063B120618400812051A7F4412052314
:0106ED0022EA
:10056B0012063B1206185002801312051A7FBE1298
:10057B000523120678AB07120678BFFF04E4FEFFD3
:10058B0022EB5401FFEBC313FBD3946340047B6357
:06059B007F01EFFEEBFF03
:0105A1002237
:10069500C2B7759852758920758DFDD28EC2B2C2CA
:0B06A500B31205A27FF47E010206B034
:1003FF00A296B3E433FFA295B3E433FEEF25E04EAC
:10040F00FFA294B3E433FEEF25E04EFFA293B3E4D3
:10041F0033FEEF25E04EFFA292B3E433FEEF25E06B
:10042F004E2414752200F523A291B3E433FFA2905A
:10043F00B3E433FEEF25E04E146010146013146024
:10044F00162403701EE52324FF8010E52324FE806D
:10045F000AE52324FD8004E52324FCF525E5223459
:10046F00FFF524AE22AF237C007D0A12035F8E229C
:0D047F008F23AE24AF2512035F8E248F253E
:01048C00224D
:10048D001206951206DD7FE87E031206B012056B8B
:10049D008E088F0985090AAF0A1206C9E50813925D
:1004AD00003000034327801205A2D2B77BFF7A06E6
:1004BD00795A850A0E1200657BFF3000067A06799F
:1004CD006080047A067964120065A299B340FBC27C
:1004DD00B7E50A75F00AA485F008F509300009247E
:1004ED0005F509E43508F5081203FFC3E509952361
:1004FD00E50895224004C2978089D3E5099525E545
:0D050D000895244003020490D29702049048
:030000000206FBFA
:0C06FB00787FE4F6D8FD75812702048D9D
:10035F00EF8DF0A4A8F0CF8CF0A428CE8DF0A42EB2
:02036F00FE226C
:10000300E51A240EF8E6051A22780B300802780E5A
:10001300E475F0011203C90203712001EB7F2ED2B4
:10002300018018EF540F2490D43440D4FF30050BD3
:10003300EF24BFB41A0050032461FFE51B600215CF
:100043001B051EE51E7002051D30080D780BE475B7
:10005300F0011203C9EF0203B70205CD7403D208FE
:100063008003E4C208F51A8B0B8A0C890DE4F51B97
:10007300F51DF51EE51B60077F2012003E80F57518
:100083001CFFC202C201C203C204C206C207C209E4
:1000930012000CFF700D3008057F0012004FAF1ED9
:1000A300AE1D22B4255FC2D5C20512000CFF24D0B9
:1000B300B40A00501A75F00A781B30D50508B6FF4C
:1000C3000106C6A426F620D5047002D20480D924E2
:1000D300CFB41A00EF5004C2E5D20502024FD20298
:1000E30080C6D20180C0D20380BCD2D580BAD206EA
:1000F30080B47F2012003E2003077401B51B00402B
:10010300F1120003FF12003E020077D209D20780EA
:1001130095120003FB120003FA120003F94A4B7015
:100123000679207A037BFF20032EE51B602A7E00DD
:100133008E8275830012038A60060EEE651C70F0D2
:10014300C2D5EBC0E0EAC0E0E9C0E0EE120296D00F
:10015300E0F9D0E0FAD0E0FB120371FF60AAEBC034
:10016300E0EAC0E0E9C0E012003ED0E02401F9D0AB
:10017300E03400FAD0E0FBE51C0460DCD51CD98038
:10018300877BFF7A027992D203809C79108002796F
:1001930008C207C2098008D2D5790A8004790AC245
:1001A300D5E51C047002F51CE4FAFDFEFF12000302
:1001B300FC7B08200213120003FD7B1030010A129E
:1001C3000003FE120003FF7B20EC3382D592D5504F
:1001D30013C3E43001069FFFE49EFEE42002039D67
:1001E300FDE49CFCE4CBF8C202EC700CCFCECDCC8A
:1001F300E824F8F870F38017C3EF33FFEE33FEED16
:1002030033FDEC33FCEB33FB994002FB0FD8E9EBF6
:10021300300205F8D0E0C448B202C0E00AEC4D4E0B
:100223004F78207B0070C2EAB51C0040BCC0E012CE
:100233000298D0F0D0E0200204C4C0E0C4B202C0EF
:10024300F0120027D0F0D5F0EB0200771203D901AA
:100253001453018E5800E54C00E14201924F019A7C
:0F02630044019A4900FA4301A0550184460184E1
:100272004501844703405000E92D00ED2E01102B6B
:1002820000F123010E2003292A00A94800000108D9
:100292003F3F3F00790AA2D5200414300609B91065
:1002A200020404B9080104A2D52007025001042067
:1002B20003689203B51B005034C0E07F203004195C
:1002C2007F30A20372077206500F1202EFC203C2FE
:1002D20007C206C2097F30800F300603E9C0E01270
:1002E200003E300603D0E0F9D0E0B51BCC30061753
:1002F2007F30B9100C12003E7F583005077F78809E
:1003020003B9080312003E3003057F2D02003E7F31
:10031200202009F87F2B2007F322920380CF286E3A
:10032200756C6C2900D2021200033002F8C2027806
:100332001B30D50108F60200A92D5043495812007E
:10034200032403B405004001E490033B9312002F01
:0D035200743A12002FD204751B0402018EB4
:10037100BB010689828A83E0225002E722BBFE028A
:09038100E32289828A83E49322BD
:10038A00BB010CE58229F582E5833AF583E0225028
:10039A0006E92582F8E622BBFE06E92582F8E22272
:0D03AA00E58229F582E5833AF583E493228C
:1003B700BB010689828A83F0225002F722BBFE0125
:0203C700F3221F
:1003C900FAE6FB0808E6F925F0F618E6CA3AF62235
:1003D900D083D082F8E4937012740193700DA3A3B3
:1003E90093F8740193F5828883E4737402936860C7
:0603F900EFA3A3A380DFC7
:1005CD00EFB40A07740D1205D8740A309811A89962
:1005DD00B8130CC2983098FDA899C298B811F6308E
:0705ED0099FDC299F5992266
:00000001FF
